:020000040800F2
:1000000048010220C1010008E9010008EB010008D5
:10001000ED010008EF010008F101000800000000F8
:10002000000000000000000000000000F3010008D4
:10003000F501000800000000F7010008751600082F
:10004000FB010008FB010008FB010008FB010008A0
:10005000FB010008FB010008FB010008FB01000890
:10006000FB010008FB010008FB010008FB01000880
:10007000FB010008FB010008FB010008FB01000870
:10008000FB010008FB010008FB010008FB01000860
:10009000FB010008FB010008FB010008B903000890
:1000A000FB010008FB010008FB010008FB01000840
:1000B0004121000871210008A5210008FB0100086A
:1000C000FB010008FB010008FB010008FB01000820
:1000D000FB010008FB01000869220008D12200088A
:1000E000FB010008FB010008FB010008FB01000800
:1000F000FB010008FB010008FB010008FB010008F0
:10010000FB010008FB010008D9210008FB010008E1
:10011000FB010008FB010008FB0100080D2200089C
:10012000FB010008FB010008FB010008FB010008BF
:10013000FB010008FB010008FB010008FB010008AF
:10014000FB010008FB010008FB010008FB0100089F
:10015000FB010008FB010008FB010008FB0100088F
:10016000FB010008FB010008FB010008FB0100087F
:10017000FB010008FB010008FB010008FB0100086F
:10018000FB010008FB010008FB010008FB0100085F
:10019000FB010008FB010008FB010008FB0100084F
:1001A00091120008FB010008FB010008DFF80CD0E9
:1001B00000F0B6F800480047593200084801022014
:1001C000DFF83800016841F470010160BFF34F8F20
:1001D000DFF82C00016821F040410160BFF36F8F10
:1001E0000848804708480047FEE7FEE7FEE7FEE7CD
:1001F000FEE7FEE7FEE7FEE7FEE7FEE788ED00E04C
:1002000034EF00E0D9200008AD0100082DE9F05FCF
:100210000546002092469B46884606468146402475
:100220001BE0284641464746224600F068F8534600
:100230005A46C01A914110D311461846224600F082
:100240004FF82D1A67EB01084F4622460120002186
:1002500000F046F817EB00094E41201EA4F10104FE
:10026000DFDC484631462A464346BDE8F09F40EA77
:1002700001039B0703D009E008C9121F08C0042A24
:10028000FAD203E011F8013B00F8013B521EF9D20B
:100290007047D2B201E000F8012B491EFBD2704733
:1002A0000022F6E710B513460A4604461946FFF742
:1002B000F0FF204610BD421C10F8011B0029FBD1A5
:1002C000801A704710B5002200E0521C835C8C5CE1
:1002D000A34201D1002BF8D1D8B2E1B2401A10BD2F
:1002E000202A04DB203A00FA02F1002070479140F6
:1002F000C2F1200320FA03F3194390407047202AEB
:1003000004DB203A21FA02F00021704721FA02F3BF
:10031000D040C2F1200291400843194670470000C6
:10032000064C074D06E0E06840F0010394E8070042
:1003300098471034AC42F6D3FFF73CFF1C3D000851
:100340003C3D000830B5144800684FF47A72B0FBA9
:10035000F2F1481EB0F1807F00D31BE0481E4FF041
:10036000E022506150170F22002807DA13071D0EF4
:100370000A4B00F00F04241F1D5503E013071C0E49
:10038000074B1C5400BF00204FF0E0229061072073
:10039000106100BF30BD00001000002018ED00E02B
:1003A00000E400E00349086000BF02490968002931
:1003B000FBD170473400002010B5402000F014F845
:1003C000012808D1402000F009F80348006810B166
:1003D00001490868804710BDC4E001200149086058
:1003E00070470000143C014001460020034A126897
:1003F0000A400AB1012000E000207047143C01408F
:1004000010B503F04FF8002010BD000070B588B0A3
:100410000646274AD2E901311068D268CDE9053194
:1004200007920490740CC6F3100000B1641C002500
:1004300009E0A54200DB0BE004A931F81500022118
:1004400000F038F86D1C04A830F815000028F0D131
:1004500000BF082C13DB0221802000F02BF80221C2
:10046000882000F027F80221902000F023F80221D4
:10047000982000F01FF80221A02000F01BF80C4B80
:1004800010330FCB8DE80F0000250AE005F10800BE
:10049000A04200DB09E03DF81500022100F00AF857
:1004A0006D1C3DF815000028F0D100BF08B070BDEC
:1004B000F03C000870B504460A460026092502B93A
:1004C00009E0012A01D1160205E0022A01D1160233
:1004D00001E04FF4407600F0F3F90546092D28D1EC
:1004E0001548006820F44070134908600846006809
:1004F000304308600846006820F0F80008600846AD
:10050000006844F0020108430B490860084600688F
:1005100040F48030086000F0D3F9054606480068D2
:1005200020F00200044908600846006820F0F80046
:100530000860284670BD0000103C02402DE9F047DD
:1005400080460E4600244FF48057A146384602F0FC
:1005500069FF04463A460021204600F0E1F80020F9
:1005600005E0215CFF2901D100212154401CB84243
:10057000F7D32068142803DDFFF742FF0020206036
:10058000002519E005EB8502211D01EBC200414663
:10059000FFF798FE78B905EB8501201D00EBC1003F
:1005A000D0F8209036B105EB8501201D00EBC1008D
:1005B000406A306003E06D1C2068A842E2DC00BFA6
:1005C000204602F011FF4846BDE8F0872DE9F041D2
:1005D00005460F464FF0000800244FF48056304681
:1005E00002F020FF044632460021204600F098F831
:1005F000002005E0215CFF2901D100212154401C8D
:10060000B042F7D32068A84209DD05EB8502201D22
:1006100000EBC2012822384602F02CFF01E04FF027
:10062000FF38204602F0E0FE4046BDE8F08170B59C
:10063000002600244FF48055284602F0F3FE0446BD
:100640002A460021204600F06BF8002005E0215CDE
:10065000FF2901D100212154401CA842F7D326686C
:10066000204602F0C1FE304670BD0000092013494B
:10067000096801F48031B1F5803F01D101201CE00F
:100680000E49096801F0100109B1062015E00B4977
:10069000096801F4807109B102200EE00749096878
:1006A00001F0E00109B1072007E00449096801F001
:1006B000020109B1082000E0092070470C3C02400B
:1006C0000348006840F0004001490860704700009E
:1006D000103C024030B502460C46092500F0F0F807
:1006E0000546092D17D10D48006820F440700B49CC
:1006F00008600846006808600846006840F001008D
:100700000860147000F0DCF805460448006820F02A
:10071000010002490860284630BD0000103C02403C
:1007200070B504460D46164632462946204602F06C
:100730004BFF002070BD2DE9F84F81460D4617464E
:100740001C464FF0000A0020009069464846FFF71B
:10075000F5FE8046B8F1000F1BD000260098401B24
:10076000A04201D20098441BA2460FE0B4F5805F7E
:1007700002D94FF4805600E0264608EB05013246C8
:100780003846FFF7CDFF3544A41B3744002CEDD18C
:1007900001E04FF0000A5046BDE8F88F05480068B8
:1007A00000F0004028B1044802490C3908600348B1
:1007B00008607047103C024023016745AB89EFCDCC
:1007C00070B504460D4626460120F0617562214849
:1007D000006810301F49024608601F4801681FA0CA
:1007E00002F0F8F9FFF7DAFF1A48006810301949EB
:1007F00002460860184801681DA002F0EBF928467F
:10080000FFF704FE134800681030124902460860E2
:10081000114801681AA002F0DDF92946204600F0CF
:1008200061F80C48006810300A49024608600A481E
:10083000016817A002F0CEF9FFF742FF05480068F3
:1008400010300449024608600348016814A002F011
:10085000C1F970BD0C00002008000020464C415337
:100860004820556E6C6F636B202E2E2E000000000A
:100870004572617365696E67202E2E2E00000000A0
:1008800050726F6772616D696E67202E2E2E0000A8
:10089000464C415348204C6F636B202E2E2E000097
:1008A00055706461746120446F6E652C20526562DE
:1008B0006F6F74204C61746572202E2E2E00000024
:1008C00008B509200090FFF7D1FE009002E0FFF785
:1008D000CDFE00909DF800000128F8D09DF80000A2
:1008E00008BD000070B505460E46002405E0295DF0
:1008F000034AA018FFF7EEFE641CB442F7D370BDA4
:100900000000020810B5024600200023102A03D17F
:100910004FF02044636E0FE0B2F5807F02D10A4CA5
:10092000236809E0B2F5805F03D1074C20342368C7
:1009300002E0054CD434236803EA01048C4201D060
:10094000002000E0012010BD840000A00021D0E9BB
:1009500000231A4383685B1E42EA4312C36842EADB
:100960004321014A11607047500100A070B5002278
:100970000021002300240568AD00A5F1C045D5F88D
:1009800040216FF30E02D0E901563543C668354366
:10099000066935434669354386693543C66935433B
:1009A000066A3543466A35432A43056835B9056802
:1009B000AD00A5F1C045C5F8402111E03B4D2B68C5
:1009C0006FF30E03D0E907563543466A35432B4390
:1009D000364D2B600568AD00A5F1C045C5F8402136
:1009E000056875BB314D0835066855F8261001F0CD
:1009F0007041856A2D686D1E866A7668761E45EAA6
:100A00000616856AAD686D1E46EA0526856AED689C
:100A10006D1E46EA0536856A2D8A6D1E46EA054634
:100A2000856AAD8A6D1E46EA0556856A2D7E6D1E65
:100A300046EA056529431D4D0835066845F8261028
:100A400032E0FFE7194D0835066855F8261001F029
:100A50007041856A2D686D1E866A7668761E45EA45
:100A60000616856AAD686D1E46EA0526856A2D8ADA
:100A70006D1E46EA054529430C4D08352C6804F0E7
:100A80007044856AED686D1E2E03856AAD8A6D1E01
:100A900046EA05552C434FF02045C5F84841034D23
:100AA0000835066845F8261070BD0000400100A01A
:100AB0000449096841EA40014FF02042C2F854114C
:100AC00070470000540100A0F0B50A460021002341
:100AD000002400BF3DE0012505FA01F3156805EA91
:100AE00003049C4234D105684F000326BE40B54341
:100AF000056015794E00B5400668354305601579E7
:100B0000012D02D01579022D16D185684F000326DC
:100B1000BE40B543856055794E00B5408668354383
:100B20008560456801268E40B543456045689679E5
:100B30008E40B6B235434560C5684F000326BE40BF
:100B4000B543C560D5794E00B540C6683543C5602C
:100B5000491C1029BFD3F0BDF0B5002300244D0778
:100B6000ED0E02FA05F3CE1000F1200555F82650DF
:100B70004E07F70E0F26BE40B543CF1000F12006FA
:100B800046F82750CE1000F1200555F8265045EACA
:100B90000304CE1000F1200545F82640F0BD418346
:100BA000704701837047000010B5FFF7CBFB01F0E1
:100BB000B9FB00F013FB01F01DFD01F00BF902F091
:100BC00053FC02F083FC09A001F036FD00240AE08A
:100BD0000A20FFF7E7FB01F06DFB18B107484FF063
:100BE00000510860641C0A2CF2DB10BD4C6F61647C
:100BF000696E67A1A3A1A3A1A30D0A00030000FFD2
:100C000030B5144B1B6903B930BD124B5B691844F6
:100C1000104B9B6919440F4B5B6A834203DC0D4BFD
:100C2000DB6A834200DAEFE70A4B9B6A8B4203DC04
:100C3000084B1B6B8B4200DAE6E74AB1054B1B8978
:100C4000044C646B034D2D6801FB050524F8153039
:100C500000BFD9E7640000201CB5012140F20F70ED
:100C600000F014FD4FF40040009003208DF80500C3
:100C700002208DF8040000208DF8060001208DF878
:100C800007000E220F21A648FFF766FF0E22002163
:100C9000A448FFF761FF0E220121A248FFF75CFF85
:100CA0000E2202219F48FFF757FF0E2203219D4885
:100CB000FFF752FF0E2204219A48FFF74DFF0E2244
:100CC00005219848FFF748FF0E2206219548FFF7B7
:100CD00043FF4FF40040009069469148FFF7F4FE4F
:100CE0000120009069468F48FFF7EEFE0220009039
:100CF00069468C48FFF7E8FE042000906946894861
:100D0000FFF7E2FE0820009069468648FFF7DCFE08
:100D10001020009069468348FFF7D6FE20200090FF
:100D200069468048FFF7D0FE4020009069467D4824
:100D3000FFF7CAFE0E2207217A48FFF70DFF0E22A9
:100D400008217848FFF708FF0E2209217548FFF7B0
:100D500003FF0E220A217348FFF7FEFE0E220B212D
:100D60007048FFF7F9FE0E2200216F48FFF7F4FEEE
:100D70000E2201216C48FFF7EFFE0E2202216A4885
:100D8000FFF7EAFE8020009069466648FFF79CFE68
:100D90004FF48070009069466248FFF795FE4FF46B
:100DA0000070009069465F48FFF78EFE4FF4806048
:100DB000009069465B48FFF787FE4FF400600090A3
:100DC00069465848FFF780FE012000906946564862
:100DD000FFF77AFE0220009069465348FFF774FE41
:100DE0000420009069465048FFF76EFE0E220C2149
:100DF0004C48FFF7B1FE0E220D214A48FFF7ACFE2A
:100E00000E2211464748FFF7A7FE0E220F21454844
:100E1000FFF7A2FE0E2203214348FFF79DFE0E229C
:100E200004214148FFF798FE0E2205213E48FFF7B6
:100E300093FE0E2206213C48FFF78EFE4FF48050B1
:100E4000009069463748FFF73FFE4FF4005000908E
:100E500069463448FFF738FE4FF4804000906946F9
:100E60003048FFF731FE4FF40040009069462D48AE
:100E7000FFF72AFE0820009069462B48FFF724FE62
:100E80001020009069462848FFF71EFE20200090A1
:100E900069462548FFF718FE402000906946224821
:100EA000FFF712FE0E2211461D48FFF755FE0E22D7
:100EB0000C211B48FFF750FE0E220D211848FFF7AA
:100EC0004BFE0E2207211848FFF746FE4FF48040E4
:100ED000009069461248FFF7F7FD4FF480500090EC
:100EE00069460F48FFF7F0FD4FF400500090694647
:100EF0000B48FFF7E9FD8020009069460A48FFF79C
:100F0000E3FD01208DF80400400300906946074886
:100F1000FFF7DAFD4FF400510448FFF742FE1CBD15
:100F2000002002400024024000280240000C024041
:100F3000F0B58FB00025032408260121880600F0B3
:100F4000D5FB0121C80500F0A1FBFFF785FE04EBEE
:100F5000C40010FB06F085B222460721284600F0A7
:100F60007BFCB00300F066FC012000F06FFC00BFCA
:100F70003D2000F03FFC0028FAD0002000900190B6
:100F8000029003900C900D900E900120049005901B
:100F900028200690082007904FF4027008904FF424
:100FA0008C70099040F20D200A904FF490700B90D5
:100FB000684600F099F90121084600F085F95820AB
:100FC0000021002807DA0A07170E1A4A00F00F035B
:100FD0001B1FD75403E00A07130E174A135400BF10
:100FE000582000F01F02012191404209920002F1B5
:100FF000E022C2F8001100BF012000F025F900F046
:1010000021F84FF4F0700D4908604FF48870486083
:101010000B48006888630A4840684863084643688C
:1010200000210268084600F045F800200349C86026
:101030000FB0F0BD18ED00E000E400E06400002017
:10104000103D000800B591B0292001904FF40270C6
:101050000290092003904FF48C70049002200590B8
:10106000FF20069000200790089009900A904FF406
:1010700080600B9005200C904FF4887010904FF01A
:1010800050400D9040F2C3300E90C01E0F9001A949
:10109000074800F0F8F90121054800F0E9F90120BE
:1010A00000F07CFA012000F0E1F811B000BD000072
:1010B000846801402DE9F04104460D4616461F465E
:1010C000064844618561A019401E0449C861E819B9
:1010D000401E086200F004F8BDE8F08164000020C2
:1010E00010B53D4901F1100201200B68002B08DB0F
:1010F000A1F114040B682468A34202DA0B681360A0
:101100000CE00B68002B02DA0023136006E0324C7F
:10111000143C0B682468A34200DB00204B68002BC2
:1011200008DB2D4C143C4B686468A34202DA4B6820
:1011300053600CE04B68002B02DA0023536006E09A
:10114000254C143C4B686468A34200DB00208B688C
:10115000002B08DB204C143C8B682468A34202DA85
:101160008B6893600FE08B68002B01DA00200AE0A7
:10117000194C143C8B682468A34204DB164B143BC7
:101180001B685B1E9360CB68002B08DB124C143C81
:10119000CB686468A34202DACB68D3600FE0CB6807
:1011A000002B01DA00200AE00B4C143CCB68646889
:1011B000A34204DB084B143B5B685B1ED3608C6866
:1011C0000B68A34203DCCC684B68A34200DD00201F
:1011D000014B143B186110BD780000201CB50121A3
:1011E000402000F053FA0121082000F04FFA0120BE
:1011F0008DF8040000208DF8060001208DF807000E
:1012000000208DF805008020009069460948FFF70E
:101210005BFC4FF48050009069460748FFF754FC90
:1012200080210448FFF7BDFC4FF480510248FFF7CE
:10123000B8FC1CBD00180240000C024001490860C7
:10124000704700003C68014030B10749096841F02F
:101250000101054A116005E00349096821F0010117
:10126000014A1160704700001868014030B1074919
:10127000096841F48031054A116005E003490968B5
:1012800021F48031014A1160704700001868014064
:1012900010B500F001F810BD10B50120FFF7CEFF2A
:1012A0000748006C01280AD1002005490864084657
:1012B000806B04490860012002498839086010BD2C
:1012C00064000020AC68014029B1064A126802435C
:1012D000044B1A6004E0034A12688243014B1A600F
:1012E0007047000034680140F0B50021002200235F
:1012F0000024002500265B4F3F68DFF86CC107EA39
:101300000C07DFF860C1CCF80070078A3904674623
:101310003F68D0F814C04CEA010C47EA0C07DFF82C
:1013200044C1CCF800700CF104073F68DFF838C105
:1013300007EA0C07DFF82CC10CF1040CCCF80070A4
:10134000078B3A0467463F68D0F81CC04CEA020C91
:1013500047EA0C07DFF80CC10CF1040CCCF8007064
:101360000CF104073F68DFF800C107EA0C07DFF85B
:10137000F4C00CF1080CCCF80070078C3B046746F5
:101380003F68D0F824C04CEA030C47EA0C07DFF8AA
:10139000D4C00CF1080CCCF800700CF104073F68C5
:1013A000DFF8C4C007EA0C07DFF8B8C00CF10C0C7A
:1013B000CCF80070078D3C046746D7F800C0C76AB8
:1013C00027434CEA070C274F0C37C7F800C03F1DD6
:1013D0003F68DFF898C007EA0C07DFF888C00CF117
:1013E000100CCCF80070D0E9007C47EA0C07D0F86C
:1013F00008C047EA0C07D0F80CC047EA0C07DFF832
:1014000064C00CF1100CDCF800C047EA0C07DFF8F0
:1014100054C00CF1100CCCF80070476B3D02078EE5
:101420003E04104F24373F6807F07F47DFF834C091
:101430000CF1240CCCF8007046EA0507D0F838C04F
:1014400047EA0C07DFF81CC00CF1240CDCF800C0E4
:1014500047EA0C07DFF80CC00CF1240CCCF8007044
:10146000F0BD00000868014000F800F08F88FE0F12
:1014700021B1026842F00102026003E0026822F03A
:101480000102026070472DE9F0410024002500268A
:10149000002200270023B1F804C04FEA0C44D0F822
:1014A00004C00CF4704CC0F804C0D1F800C04CEA81
:1014B000040CC0F804C0B1F80CC04FEA0C45D0F8D9
:1014C00008C00CF4704CC0F808C0D1F808C04CEA51
:1014D000050CC0F808C0D0F810C02CF0070CC0F8FC
:1014E00010C0D1F810C0C0F810C0D1F81CC04FEA2D
:1014F0000C26B1F820C04FEA0C4291F824C04FEA04
:101500000C67D0F818C09C46C0F818C0D1F818C0B5
:101510004CEA060C4CEA020C4CEA070CC0F818C066
:10152000D0F814C02CF0FF0CC0F814C0D1F814C0CF
:10153000C0F814C0D0F81CC040F207782CEA080CA0
:10154000C0F81CC0D1E90AC84CEA080CC0F81CC09D
:10155000D0F828C09C46C0F828C0D1F830C0C0F8E8
:1015600028C0B1F838C04FEA0C43D0F82CC00CF0BA
:10157000E02CC0F82CC0D1F834C04CEA030CC0F801
:101580002CC0D0F830C06FF30A0CC0F830C0D1F8CE
:101590003CC0C0F830C0BDE8F081000001490860DF
:1015A000704700002468014070B5002100230F221D
:1015B000C4781CB3174C246804F4E064C4F5E064F8
:1015C000C4F30721C1F10404E3B20A4144789C400A
:1015D000E1B28478144021430C07210E0E4C0578AB
:1015E0006155047804F01F050124AC4005786D11A5
:1015F000AD0005F1E025C5F8004109E0047804F0EC
:101600001F050124AC40054D0678761145F82640AB
:1016100070BD00000CED00E000E400E080E100E0BF
:10162000024A0A400243024B1A60704780FFFF1FC4
:1016300008ED00E000BF00BF00BFBFF34F8F00BF49
:1016400000BF00BF0948006800F4E0600849084393
:10165000001D0649086000BF00BF00BFBFF34F8FE9
:1016600000BF00BF00BF00E000BFFDE70CED00E0E1
:101670000000FA050448006820B103480068401ED5
:1016800001490860704700003400002029B1064A73
:1016900012680243044B1A6004E0034A1268824352
:1016A000014B1A60704700003038024029B1064AE9
:1016B00012680243044B1A6004E0034A1268824332
:1016C000014B1A60704700003838024029B1064AC1
:1016D00012680243044B1A6004E0034A1268824312
:1016E000014B1A60704700004038024029B1064A99
:1016F00012680243044B1A6004E0034A12688243F2
:10170000014B1A607047000044380240F0B50021D8
:1017100000220024022500260223324F3F6807F0F2
:101720000C0121B1042905D0082937D105E02E4F3D
:10173000076036E02D4F076033E02A4F3F1F3F68B8
:10174000C7F38056274F3F1F3F6807F03F036EB136
:10175000264FB7FBF3F7DFF88CC0ACF1040CDCF8D4
:1017600000C0CCF3881C07FB0CF40CE01E4FB7FB49
:10177000F3F7DFF870C0ACF1040CDCF800C0CCF378
:10178000881C07FB0CF4174F3F1F3F68C7F3014746
:101790007F1C7D00B4FBF5F7076002E0124F076085
:1017A00000BF00BF0F4F3F6807F0F0010909104F5D
:1017B0007A5C0768D74047600A4F3F6807F4E051FA
:1017C000890A0B4F7A5C4768D7408760054F3F68AE
:1017D00007F46041490B064F7A5C4768D740C76001
:1017E000F0BD0000083802400024F40040787D017C
:1017F0002400002010B501460022002300204A11D9
:10180000012A02D10A4C236808E0022A03D1084CBD
:101810007034236802E0064C7434236801F01F0220
:10182000012494401C400CB1012000E0002010BDB8
:101830000038024001460020034A106820F440307E
:1018400008431060704700008C3802400149086767
:10185000704700000000474210B5830143EA01636E
:1018600043EA0273014C236010BD00008838024037
:101870001CB501214FF4FE70FFF708FF02208DF820
:10188000040003208DF8050000208DF806008DF877
:1018900007000C220021FE48FFF75EF90C2201210F
:1018A000FB48FFF759F90C220221F948FFF754F9D8
:1018B0000C220321F648FFF74FF90C220421F448CB
:1018C000FFF74AF90C220521F148FFF745F90C22F0
:1018D0001146EF48FFF740F90C220D21EC48FFF7C5
:1018E0003BF90C220E21EA48FFF736F90C220F21B2
:1018F000E748FFF731F90C220021E648FFF72CF901
:101900000C220121E348FFF727F9012000906946E6
:10191000DF48FFF7D9F8022000906946DC48FFF75E
:10192000D3F8042000906946D948FFF7CDF8082085
:1019300000906946D648FFF7C7F810200090694626
:10194000D348FFF7C1F8202000906946D048FFF740
:10195000BBF84FF4805000906946CD48FFF7B4F8CB
:101960004FF4005000906946C948FFF7ADF84FF4B6
:10197000804000906946C648FFF7A6F84FF4004043
:1019800000906946C248FFF79FF801200090694621
:10199000C048FFF799F8022000906946BD48FFF75C
:1019A00093F80C220E21BC48FFF7D6F80C220F2129
:1019B000B948FFF7D1F80C220021B748FFF7CCF85F
:1019C0000C220121B448FFF7C7F80C220721B348C5
:1019D000FFF7C2F80C220821B048FFF7BDF80C222F
:1019E0000921AE48FFF7B8F80C220A21AB48FFF7EF
:1019F000B3F80C220B21A948FFF7AEF80C221146D0
:101A0000A648FFF7A9F80C220D21A448FFF7A4F877
:101A10000C220E21A148FFF79FF80C220F219F48AE
:101A2000FFF79AF80C2208219B48FFF795F80C2243
:101A300009219948FFF790F80C220A219648FFF7F0
:101A40008BF80C2208219648FFF786F80C22092112
:101A50009348FFF781F80C220A219148FFF77CF8A0
:101A60000C220B218E48FFF777F80C2211468C4888
:101A7000FFF772F80C220D218948FFF76DF80C2250
:101A80000E218748FFF768F80C220F218448FFF7E2
:101A900063F80C2200218348FFF75EF80C22012135
:101AA0008048FFF759F80C2202217E48FFF754F8CE
:101AB0000C2203217B48FFF74FF80C2206217948BE
:101AC000FFF74AF80C2207217648FFF745F80C2269
:101AD00009217448FFF740F80C220A217148FFF7EA
:101AE0003BF84FF48040009069466B48FEF7ECFFEE
:101AF0004FF40040009069466748FEF7E5FF01207B
:101B0000009069466448FEF7DFFF022000906946B6
:101B10006148FEF7D9FF8020009069465F48FEF7D4
:101B2000D3FF4FF48070009069465C48FEF7CCFF0D
:101B30004FF40070009069465848FEF7C5FF4FF417
:101B40008060009069465548FEF7BEFF4FF4006084
:101B5000009069465148FEF7B7FF4FF4805000905F
:101B600069464E48FEF7B0FF4FF4005000906946BA
:101B70004A48FEF7A9FF4FF4804000906946474865
:101B8000FEF7A2FF4FF40040009069464348FEF77D
:101B90009BFF4FF48070009069463F48FEF794FF2A
:101BA0004FF40070009069463B48FEF78DFF4FF4FC
:101BB0008060009069463848FEF786FF4FF48070D9
:101BC000009069463648FEF77FFF4FF400700090A2
:101BD00069463348FEF778FF4FF48060009069460D
:101BE0002F48FEF771FF4FF40060009069462C48C3
:101BF000FEF76AFF4FF48050009069462848FEF7D0
:101C000063FF4FF40050009069462548FEF75CFFE3
:101C10004FF48040009069462148FEF755FF4FF48D
:101C20000040009069461E48FEF74EFF01200090DC
:101C300069461C48FEF748FF022000906946194893
:101C4000FEF742FF0420009069461648FEF73CFF6D
:101C50000820009069461348FEF736FF40200090A8
:101C600069461048FEF730FF8020009069460D4815
:101C7000FEF72AFF4FF40070009069460948FEF70E
:101C800023FF4FF480600090694606480CE0000096
:101C90000014024000180240000C024000100240F4
:101CA000001C024000200240FEF70EFF0C2206211D
:101CB0004248FEF751FF0C2204214148FEF74CFF39
:101CC0000C2205213E48FEF747FF0C2200213D482B
:101CD000FEF742FF0C220B213B48FEF73DFF0C2292
:101CE0000F213748FEF738FF0C2208213448FEF751
:101CF00033FF0C2207213148FEF72EFF0C22012171
:101D00003248FEF729FF0C2200213048FEF724FF5D
:101D10000C2204212E48FEF71FFF0C2205212C481F
:101D2000FEF71AFF4020009069462448FEF7CCFEDB
:101D30001020009069462248FEF7C6FE2020009041
:101D400069461F48FEF7C0FE0120009069461D4805
:101D5000FEF7BAFE4FF40060009069461A48FEF79D
:101D6000B3FE4FF40040009069461548FEF7ACFE04
:101D70004FF48070009069461148FEF7A5FE802060
:101D8000009069460D48FEF79FFE022000906946CC
:101D90000E48FEF799FE0120009069460B48FEF7B9
:101DA00093FE1020009069460948FEF78DFE202022
:101DB000009069460648FEF787FE1CBD001C0240E5
:101DC00000180240000802400014024000100240C7
:101DD0000020024010B592B0002401210846FFF710
:101DE00065FCFFF745FD02200090072001900420CC
:101DF0000290062003900220049005900690012096
:101E00000790002008900420099020200A9040208C
:101E10000B904FF4C0700C9000200D904FF40060B8
:101E20000E9040000F9040001090CDF844D007A8CD
:101E3000FEF79CFD00F019F800BF06E04FF05531A9
:101E4000A000A0F140500160641CB4F5800FF5D3F0
:101E5000002405E00021A000A0F140500160641CB6
:101E6000B4F5800FF6D312B010BD1FB500240120C9
:101E7000009008200190012002900020039000BFF4
:101E800020210120FEF73EFD0028F9D16846FEF72B
:101E90005DFD012000F046F802200090082001902E
:101EA000012002900020039002E06846FEF74EFDFC
:101EB00020210120FEF726FD0028F6D1012000F0A8
:101EC00031F8032000900820019002900020039038
:101ED00000BF20210120FEF715FD0028F9D168463A
:101EE000FEF734FD40F231240420009008200190D8
:101EF00001200290039400BF20210120FEF702FD83
:101F00000028F9D16846FEF721FD40F26A50FEF73D
:101F1000CFFD00BF20210120FEF7F4FC0028F9D1FD
:101F20001FBD000001B581B0002000900549019857
:101F30004843009002E00098401E0090009800285E
:101F4000F9D10CBDA086010021B1028842F0400207
:101F5000028004E002884FF6BF731A400280704787
:101F60000246002013890B400BB1012000E0002045
:101F700070470146888970478181704710B50022FB
:101F8000028802F441520B884C8823438C882343F7
:101F9000CC8823430C8923434C8923438C892343D6
:101FA000CC8923431A430280838B4FF2FF74234072
:101FB00083830B8A038210BD0CB500200190009032
:101FC0004148006840F480303F49086000BF3E4807
:101FD000006800F4003000900198401C01900098C7
:101FE00018B90198B0F5A04FF1D13748006800F456
:101FF000003010B10120009001E000200090009816
:10200000012860D130484030006840F080502E49AF
:10201000403108602D48006840F440402B4908607A
:1020200029480830006828490831086008460068D7
:1020300040F4004008600846006840F4A050086082
:102040002348091F0860081F006840F08070091FBE
:10205000086000BF1C48006800F000700028F9D03C
:102060001A48006840F480301849086000BF1748DB
:10207000406800F480300028F9D01448006840F42B
:1020800000301249086000BF1048406800F400307A
:102090000028F9D040F205700E4908600A4808305F
:1020A000006820F00300084908310860084600680D
:1020B00040F00200086000BF03480830006800F0EC
:1020C0000C000828F8D10CBD003802400070004018
:1020D000195A4007003C024010B51548006840F40A
:1020E0007000134908601348006840F0010011496E
:1020F000086000200F49083108600E4800680E494A
:1021000008400C4908600D48091D0860081F006858
:1021100020F48020091F0860002006490C31086067
:10212000FFF74AFF4FF0006001498039086010BD99
:1021300088ED00E000380240FFFFF6FE103000247A
:1021400070B54FF0804400250121204600F07BF857
:1021500001280AD105480078012802D103494868BE
:1021600080470121204600F06BF870BDD8E00120C7
:1021700070B50A4C01250121204600F064F80128C1
:102180000AD10748007A012802D10549C86880476A
:102190000121204600F054F870BD0000000400400A
:1021A000D8E0012070B50A4C02250121204600F03C
:1021B0004AF801280AD10748007C012802D10549C4
:1021C000486980470121204600F03AF870BD0000C0
:1021D00000080040D8E0012070B50A4C0325012119
:1021E000204600F030F801280AD10748007E012877
:1021F00002D10549C86980470121204600F020F836
:1022000070BD0000000C0040D8E0012070B50A4C01
:1022100005250121204600F016F801280BD10748BA
:1022200090F82800012802D10449C86A804701219A
:10223000204600F005F870BD00140040D8E00120F1
:10224000CA430282704730B50246002000230024B2
:10225000158A05EA0103958905EA010413B10CB159
:10226000012000E0002030BD10B500240E48008899
:1022700000F0200078B10C48001D0088C4B221464F
:102280000A4800F043FC0A48006858B12046084953
:102290000968884706E004480088C4B20248001D67
:1022A0000088C4B210BD00000044004020E10120BD
:1022B0005C000020014908787047000038000020C9
:1022C000024908780021014A117070473A00002045
:1022D00010B5002440F225510E4800F0C8F8B8B1FE
:1022E0000C4800F07DF90C4908700C48007809781A
:1022F00048400A490978084030B108480078064942
:102300000978484006490870034800780349087076
:1023100010BD0000004800403800002039000020B7
:102320003A00002000B587B001210220FFF7AEF986
:1023300002208DF8180000208DF81A0001208DF879
:102340001B0000208DF819004FF48060059005A94E
:102350002248FEF7B9FB4FF40060059005A91F481D
:10236000FEF7B2FB07220A211C48FEF7F5FB072205
:102370000B211A48FEF7F0FB01218804FFF7A6F9AC
:102380004FF4E13001900020ADF80800ADF80A00EC
:10239000ADF80C000C20ADF80E000020ADF81000D8
:1023A00001A90F4800F0B2F827208DF800000320A3
:1023B0008DF801008DF8020001208DF803006846B9
:1023C000FFF7F2F80121064800F00CF8012240F274
:1023D0002551034800F075F807B000BD0004024025
:1023E0000048004021B1828942F40052828104E019
:1023F00082894DF6FF731A40828170471CB5012116
:102400000846FFF743F902208DF8040000208DF8FC
:10241000060001208DF8070000208DF805004FF41C
:102420000070009069460A48FEF74EFB4FF480604A
:10243000009069460648FEF747FB07220921044839
:10244000FEF78AFB07220A210148FEF785FB1CBD27
:102450000000024002460020B1F5007F00D100BF1D
:1024600013880B400BB1012000E00020704770B5CD
:102470000246002400230025002040F66A16B142DF
:1024800000D100BFC1F3421501F01F03012606FA77
:1024900003F3012D02D19689334006E0022D02D1CB
:1024A000168A334001E0968A33400C12012606FA60
:1024B00004F41688344013B10CB1012000E0002070
:1024C00070BDF0B50346002400260025002040F62C
:1024D0006A17B94200D100BF1846C1F3421401F097
:1024E0001F06012707FA06F5012C01D10C3004E084
:1024F000022C01D1103000E014301AB107682F43CC
:10250000076002E00768AF430760F0BD2DE9FF47B1
:1025100005460E460024A14600BFA046B08900B182
:1025200000BF2C8A24F44054F08804432C82AC89E8
:1025300041F20C608443B0883189084371890843B3
:102540000443AC81AC8A24F44074B0890443AC8267
:102550006846FFF7DBF82048854202D01F488542D5
:1025600002D1DDF80C9001E0DDF80890A88900F4B4
:10257000004040B109EBC90000EB09103168490087
:10258000B0FBF1F707E009EBC90000EB0910316877
:102590008900B0FBF1F76420B7FBF0F004012009DB
:1025A000642101FB1078A88900F4004040B132207A
:1025B00000EBC800B0FBF1F000F00700044308E0B6
:1025C000322000EB08106421B0FBF1F000F00F00A6
:1025D00004432C81BDE8FF87001001400014014036
:1025E00001468888C0F308007047C1F30802828062
:1025F000704700001FB501211020FFF777F8FFF7A3
:10260000FDFE4FF4E13000900020ADF80400ADF87D
:102610000600ADF808000C20ADF80A000020ADF867
:102620000C0069460348FFF771FF01210148FFF7DD
:10263000D9FE1FBD001001400FB4054B10B503A912
:10264000044A029800F02CF810BC5DF814FB00005E
:10265000412D0008600000200FB4084B10B504A9FC
:1026600002AA039800F01CF8044602A9002000F01A
:1026700048FA204610BC5DF814FB0000032B00084C
:1026800002E008C8121F08C1002AFAD1704770473B
:10269000002001E001C1121F002AFBD17047000099
:1026A0002DE9FF4F8DB00F460546002606E0252890
:1026B0000BD0DDE90F1290476D1C761C287800289E
:1026C000F5D111B03046BDE8F08F0024A246A146F6
:1026D0000122EC4900E0044315F8013F203B02FAD7
:1026E00003F00842F7D128782A2810D06FF02F0283
:1026F0002878A0F13001092914D80AEB8A0102EBED
:10270000410144F0020400EB010A6D1CF0E701CF27
:102710005FEA000A03D544F40054CAF1000A44F009
:1027200002046D1C28782E2817D115F8010F44F0EB
:1027300004042A280ED06FF02F022878A0F130016F
:1027400009290AD809EB890102EB410100EB0109D3
:102750006D1CF2E757F8049B6D1C28786C280FD08D
:1027600006DC4C2817D068280DD06A2814D104E064
:10277000742810D07A280FD10DE044F400140AE038
:1027800044F4801401E044F440146978814202D199
:1027900004F580146D1C6D1C2A786E2A1FD00CDC89
:1027A000632A31D004DC002A8BD0582A11D1A3E04F
:1027B000642A68D0692A0CD165E0732A2ED004DC23
:1027C0006F2A73D0702A04D19BE0752A6FD0782AC3
:1027D0006ED01046DDE90F129047761C50E1C4F32D
:1027E0000250022806D0032809D0042801CF09D0BE
:1027F000066045E101CFF117C0E9006140E101CF7A
:1028000006803DE106703BE117F8040B8DF80000EF
:1028100000208DF80100EB46012003E057F804BBCF
:102820004FF0FF3061074FF0000102D40DE008F1D6
:102830000101884649450FDA8045F8DB1BF808108E
:102840000029F4D108E008F1010188468142FADB51
:102850001BF808100029F6D1DDE90F23AAEB0800C8
:102860008146214600F036F9304400EB080604E0CA
:10287000DDE90F121BF8010B9047B8F10108F7D200
:1028800021464846F7E00A21C4F302534FF0000BFB
:102890000891022B04D001CFC117032B09D00AE005
:1028A000FF1D27F00707F7E8020108E032E01FE00C
:1028B00020E000B2C117042B01D140B2C117031EA2
:1028C00071F1000307DA4FF0000CD0EB0C006CEB59
:1028D00001012D2302E0230504D52B238DF824309C
:1028E000012303E0E30701D02023F7E7984658E0EF
:1028F0000A2110E010210EE010204FF0000B08908C
:102900000CE010214FF0000B44F004044FF00809D4
:10291000089103E008214FF0000B0891C4F3025323
:10292000022B04D001CF0021032B06D006E0FF1DAF
:1029300027F00707F7E8020103E080B2042B00D17B
:10294000C0B24FF0000823072BD5702A07D0DDF85E
:1029500020C08CF0100C5CEA0B0C05D00EE040237C
:102960008DF82430012308E050EA010306D030231B
:102970008DF824308DF8252002239846DDF820C0FC
:102980008CF0080C5CEA0B0C0BD150EA010301D16E
:10299000630706D530238DF824304FF00108A9F1E4
:1029A0000109582A04D038A20B9208AA0A920BE017
:1029B0003AA2F9E75B46089AFDF728FC0B9B9B5C63
:1029C0000A9A521E0A92137050EA0102F2D10A9832
:1029D000ADEB000000F1200B600702D524F4803439
:1029E00001E04FF00109D94502DDA9EB0B0000E041
:1029F000002000EB0B0141440890AAEB010AE00320
:102A000006D4DDE90F232146504600F063F8064462
:102A10004FF0000908E009A911F80900DDE90F12DB
:102A2000904709F10109761CC145F4DBE0030CD5A0
:102A3000DDE90F232146504600F04CF8064404E03F
:102A4000DDE90F1230209047761C0899481E089047
:102A50000029F5DC08E00A980A990078491C0A91D7
:102A6000DDE90F129047761CBBF10001ABF1010BC1
:102A7000F1DC21465046DDE90F2300F019F8064449
:102A80006D1C1BE6092801003031323334353637EE
:102A900038396162636465660000000030313233AA
:102AA000343536373839414243444546000000004A
:102AB0002DE9F041044600251E461746880404D43B
:102AC00005E039462020B0476D1C641EF9D5284624
:102AD000BDE8F0812DE9F041044600251E469046F0
:102AE000C80301D5302700E02027880404D505E07D
:102AF00041463846B0476D1C641EF9D52846BDE8EE
:102B0000F0810A68531C0B601070704710B50246C4
:102B100012B94FF0FF3010BD4FF0FF33106910B104
:102B20005069884201D101201062D2E90040A042E0
:102B30001BDA106AC8B1D468506A01555068401C4D
:102B40005060106938B19069884204D1D069401C46
:102B5000D06100201062D068401CD0601468D0683A
:102B6000A04201DB0020D06000231846D3E700001C
:102B70002DE9F0418CB006460F469046302168465C
:102B8000FDF78EFB002008E0A6F12001104A02EBC1
:102B90000111095C0DF80010401C1028F4DB002422
:102BA0000FE000250AE01DF80430AB4003F080027E
:102BB00008EB04017819FEF723F86D1C082DF2DBF1
:102BC000641C102CEDDB08200CB0BDE8F081000087
:102BD0000037000870B504460D46164604B970BDAE
:102BE0000AE0207800F0800030B92078324629468B
:102BF000FFF7BEFF0544641C20780028F1D100BF18
:102C0000EDE7000070B501461148007A08B90120CF
:102C100070BD00200F4BD3E900430C1B984114D228
:102C20000D480068B1FBF0F30948406830F81340E4
:102C3000002206E00020064D6D689E1825F816005B
:102C4000521CA242F6D30020E2E70220E0E7000097
:102C5000AC000020480000204400002000B54EF2E7
:102C60004860124908604FF48070114908601149AA
:102C70000020114AC2E900101048114908601148AB
:102C8000486000200872094909684A000C494868F0
:102C9000002100F0FCFB0A49086807490A68002186
:102CA00000F0F5FB01200649087200BD400000203D
:102CB00044000020694BE6004800002090B419D081
:102CC000AC00002000E817D0F0B503460021002535
:102CD0000BB9481EF0BD17480068B3FBF0F2154869
:102CE0000068B3FBF0F600FB163000B1521C12482E
:102CF0000068411E19E01148406830F8110008B919
:102D00006D1C00E0002595420ED1002405E00B4E1D
:102D100076680F1926F81720641C9442F7D3054EE5
:102D2000366801FB06F0D5E7491E0029E3DA4FF0CB
:102D3000FF30CFE74400002040000020AC0000201E
:102D400038B504468DF8000069460320ABBE204626
:102D500038BD00002DE9F04F8BB0FEF7E9F8FEF723
:102D600071F95C48006810305A49024608605A48B8
:102D700001685AA0FFF72EFF5648006810305549E9
:102D8000024608605448016858A0FFF723FF5148E5
:102D9000006810304F49024608604F48016857A04C
:102DA000FFF718FFFDF743FC06464FF4807000F074
:102DB00039FB0A90B00000F035FB07464FF00008E1
:102DC00000252AE028216846FDF76AFA6946284668
:102DD000FDF7FCFB6846FDF76EFA8346ABF1040194
:102DE0006A4688184CA1FDF76DFAA8B908F10202ED
:102DF0006B464BA10A98FFF72FFC47F8285008F1C3
:102E000001083448006810303249024608603248F0
:102E100001680A98FFF7DEFE6D1CB542D2DB0FF2A7
:102E2000181A002406F102092A48006810302949BE
:102E300002460860284801685046FFF7CBFE3DE097
:102E4000FFF73EFA054622463FA10A98FFF704FC29
:102E50005046FDF730FA2049096801EBC00B1D48C8
:102E6000594602680A98FFF7B5FE102D06D1002CCE
:102E700001DD641E21E0A9F101041EE0202D07D12F
:102E8000A9F10100A04201DD641C16E0002414E059
:102E9000042D12D104B912E0012C04D12C484107B1
:102EA0000860FEF7C7FB2A48401C01070860A01E07
:102EB00057F820004860FEF7BDFB00BFC0E700BF29
:102EC0000A9800F091FA384600F08EFA0BB0BDE88F
:102ED000F08F00000C00002008000020506C65619D
:102EE00073652053656C6563743A000030302E20A2
:102EF000426F6F74204E6F770000000030312E203B
:102F000055706461746120757365722E61707020F4
:102F100046696C65000000002E61707000000000C2
:102F2000253032642E205570646174612025732031
:102F300046696C6500000000596F75722053656C1E
:102F40006563742069733A00253032640000000024
:102F5000010000FF2DE9F843FDF7EAFFFEF772F8E4
:102F6000294800681030284902460860274801684F
:102F700027A0FFF72FFE0020009000268046224861
:102F8000006810302049024608602048016824A0EB
:102F9000FFF720FE694627A0FDF7D0FA064609256F
:102FA0000099481900F03EFA0446CEB122460021AD
:102FB00020A0009BFDF7BFFB0099884210D100992B
:102FC00060182A461BA1FDF752F927461C490098B4
:102FD00008443862009841192046FDF7F1FB0AE0E9
:102FE000094800681030084902460860074801682F
:102FF00014A0FFF7EFFD204600F0F6F942F2107042
:10300000FDF7D0F9BDE8F8830C000020080000208F
:10301000496E697420446F6E65202E2E2E000000CC
:1030200046696E6420757365722E6170702E2E2E47
:1030300000000000757365722E6170700000000062
:103040000000020843616E27742046696E64207593
:103050007365722E6170702C205265626F6F7420E0
:103060004C61746572202E2E2E0000002DE9F04771
:103070008AB0FDF75DFFFDF7E5FF4FF4807000F0CB
:10308000D1F9824642480068103041490246086042
:103090004048016840A0FFF79DFD0024A046A146DE
:1030A00028216846FDF7FCF84FF000503EA1426829
:1030B0005046FFF7D1FA36480068103034490246CE
:1030C0000860344801685046FFF784FD4FF0005116
:1030D00048686946FDF77AFA002831D16A4639A175
:1030E0005046FFF7B9FA2A480068103028490246CE
:1030F0000860284801685046FFF76CFDDDF8208025
:10310000099C6846FDF7D7F8461CA01900F08AF91B
:10311000054623462A4600216846FDF70CFB281980
:1031200032466946FDF7A3F82F462B482044386203
:10313000A1192846FDF744FB284600F055F91CE08C
:103140004FF0005025A142685046FFF785FA10481D
:10315000006810300E49024608600E48016850466B
:10316000FFF738FD0A480068103009490246086038
:103170000848016821A0FFF72DFD504600F034F902
:1031800042F21070FDF70EF90AB0BDE8F0870000BA
:103190000C00002008000020496E697420446F6E06
:1031A00065202E2E2E00000046696E642046696C54
:1031B0006520427920496E6465782025642E2E2E84
:1031C0000000000046696C65204E616D65206973E2
:1031D0003A2025732E2E2E000000020843616E2730
:1031E000742046696E642046696C652042792049E6
:1031F0006E6465782025642E2E2E00005265626F65
:103200006F74204C61746572202E2E2E0000000019
:1032100010B50E4800680E490840B0F1005F0DD1AE
:103220004FF400318802FEF7FBF908484468014674
:10323000086880F3088800BFA04705E005484FF004
:1032400000510860FEF7F6F910BD0000000002080A
:103250000000F02F030000FFFDF7A6FC4FF0005028
:1032600000681049884202D1FFF774FD12E04FF068
:10327000005000680B49891E884202D1FFF76AFEA0
:1032800008E04FF0005000680649491E884201D10D
:10329000FFF7ECFE00204FF000510860FFF7B8FF89
:1032A00000BFFEE7030000FF70B501461148007A39
:1032B00008B9012070BD00200F4BD3E900430C1B5F
:1032C000984114D20D480068B1FBF0F309484068FA
:1032D00030F81340002206E00020064D6D689E186D
:1032E00025F81600521CA242F6DB0020E2E702207D
:1032F000E0E70000B8E00120480000205400002072
:1033000000B540F61C601149086020201049086093
:103310001048114908601148114908601148486077
:1033200000200872094909684A000D4948680021CF
:1033300000F0ADF80A49086807490A68002100F062
:10334000A6F801200649087200BD000050000020C8
:1033500054000020C3C3010058000020F01C0020CE
:10336000B8E00120B800002070B503460021002518
:103370000BB9481E70BD19480068B3FBF0F082B26B
:1033800016480068B3FBF0F600FB163008B1501C7D
:1033900082B213480068411E1AE01248406830F8B3
:1033A000110010B9681C85B200E0002595420ED1CD
:1033B000002405E00B4840680E1920F81620641C14
:1033C0009442F7D3054E366801FB06F0D2E7491E5A
:1033D0000029E2DA4FF0FF30CCE700005400002073
:1033E00050000020B8E0012070B50446264604B91C
:1033F00070BD06F07040B0F1005F06D1074800686C
:10340000251A2846FFF750FF05E005480068251AF1
:103410002846FFF7F7FB00BFEAE70000B8E001200D
:10342000AC00002070B505460026B5F5A05F01D9B7
:10343000741E03E02846FFF797FF0446601C18B18E
:1034400007480068061908E02846FFF73DFC0446D7
:10345000601C10B1034800680619304670BD0000BA
:10346000B8E00120AC00002010B5FFF749FFFFF7DE
:10347000F5FB10BD70B503460C4603E014F8015B84
:1034800003F8015B1500A2F10102F7D170BD30B560
:10349000034601E003F8011B1400A2F10102F9D177
:1034A00030BD000010B500F0EDF808210648FDF72A
:1034B00076FBC72000F0B0F808210348FDF771FB48
:1034C00000F0C6F810BD00000018024000B585B03D
:1034D00000F02EF808211448FDF763FB0020ADF83A
:1034E00000004FF48270ADF802000020ADF8040037
:1034F0000220ADF806000120ADF808004002ADF84A
:103500000A000020ADF80C00ADF80E000720ADF861
:10351000100069460548FEF731FD01210348FEF71A
:1035200013FD05B000BD000000180240003001404E
:103530001CB501210803FEF7D9F801214220FEF74E
:10354000A5F8052203211E48FDF706FB05220421EC
:103550001B48FDF701FB052211461948FDF7FCFA4F
:1035600002208DF804008DF8050000208DF806007B
:1035700002208DF807000820009069461048FDF7EA
:10358000A3FA2020009069460D48FDF79DFA10200F
:10359000009069460A48FDF797FA0820009001203C
:1035A0008DF8040000208DF8060002208DF805003B
:1035B00000208DF8070069460248FDF785FA1CBD1A
:1035C000000402400018024070B505460C4616463D
:1035D00008211048FDF7E3FA032000F01DF8C4F3BA
:1035E000074000F019F8C4F3072000F015F8E0B226
:1035F00000F012F804E0A52000F00EF828706D1C11
:103600003000A6F10106F6D108210248FDF7C9FAFB
:1036100070BD00000018024010B5044600BF022132
:103620000A48FEF79DFC0028F9D021460748FEF71E
:10363000A3FC00BF01210548FEF792FC0028F9D049
:103640000248FEF796FCC0B210BD000000300140F9
:1036500010B5002408210A48FDF7A1FA0520FFF75C
:10366000DBFF00BFA520FFF7D7FF044604F00100F1
:103670000028F7D108210248FDF793FA10BD000099
:103680000018024010B508210548FDF788FA062009
:10369000FFF7C2FF08210248FDF783FA10BD0000C2
:1036A00000180240002070470020704710B5044603
:1036B000E1B20648FEF799FF00BF80210348FEF7FC
:1036C000C9FE0028F9D0204610BD000000100140BE
:1036D00070B506460C4600250BE0715D0748FEF705
:1036E00084FF00BF80210548FEF7B4FE0028F9D012
:1036F0006D1CA542F1DB204670BD000000100140AA
:1037000000000000000000000000000000000000B9
:103710000000001010101010101000001818000009
:1037200000123624480000000000000000000000E5
:10373000000000242424FE484848FE484848000071
:1037400000001038545450301814145454381010C9
:1037500000000044A4A8A8A8541A2A2A2A44000059
:1037600000000030484848506EA4948889760000D4
:1037700000606020C00000000000000000000000A9
:1037800000020408081010101010100808040200AD
:1037900000402010100808080808081010204000F9
:1037A000000000001010D63838D6101000000000BD
:1037B0000000000010101010FE101010100000008B
:1037C000000000000000000000000000606020C059
:1037D00000000000000000007F000000000000006A
:1037E0000000000000000000000000006060000019
:1037F00000000102020404080810102020404000CC
:103800000000001824424242424242422418000072
:10381000000000107010101010101010107C00002C
:103820000000003C4242420404081020427E000096
:103830000000003C424204180402024244380000E6
:10384000000000040C14242444447E04041E0000E0
:103850000000007E404040586402024244380000AC
:103860000000001C244040586442424224180000DA
:103870000000007E444408081010101010100000D2
:103880000000003C4242422418244242423C0000D4
:103890000000001824424242261A02022438000086
:1038A00000000000000018180000000018180000B8
:1038B00000000000000000100000000000101020B8
:1038C000000000020408102040201008040200003C
:1038D000000000000000FE000000FE0000000000EC
:1038E00000000040201008040204081020400000DE
:1038F0000000003C42426202040808001818000060
:1039000000000038445AAAAAAAAAB44244380000C7
:103910000000001010182828243C444242E7000010
:10392000000000F8444444784442424244F8000015
:103930000000003E42428080808080424438000087
:10394000000000F8444242424242424244F8000031
:10395000000000FC424848784848404242FC0000D1
:10396000000000FC424848784848404040E00000E1
:103970000000003C44448080808E84444438000031
:10398000000000E7424242427E42424242E70000DB
:103990000000007C1010101010101010107C00009F
:1039A0000000003E0808080808080808080888F011
:1039B000000000EE444850705048484444EE000077
:1039C000000000E0404040404040404042FE0000D7
:1039D000000000EE6C6C6C6C5454545454D60000CF
:1039E000000000C7626252524A4A4A4646E200005C
:1039F0000000003844828282828282824438000041
:103A0000000000FC424242427C40404040E0000056
:103A100000000038448282828282B2CA4C3806009A
:103A2000000000FC4242427C4848444442E300001B
:103A30000000003E4242402018040242427C000046
:103A4000000000FE9210101010101010103800002E
:103A5000000000E74242424242424242423C0000F1
:103A6000000000E7424244242428281810100000D7
:103A7000000000D692929292AAAA6C44444400009C
:103A8000000000E7422424181818242442E700000C
:103A9000000000EE444428281010101010380000D8
:103AA0000000007E840408081020204242FC000030
:103AB000001E1010101010101010101010101E000A
:103AC00000004040202010101008080404040202E6
:103AD0000078080808080808080808080808780096
:103AE000001C220000000000000000000000000098
:103AF000000000000000000000000000000000FFC7
:103B00000060100000000000000000000000000045
:103B1000000000000000003C421E2242423F000024
:103B2000000000C0404040586442424264580000D7
:103B3000000000000000001C22404040221C000049
:103B4000000000060202021E22424242261B000022
:103B5000000000000000003C427E4040423C00006B
:103B60000000000F1110107E10101010107C0000CB
:103B7000000000000000003E444438403C42423C0B
:103B8000000000C04040405C6242424242E7000008
:103B9000000000303000007010101010107C000089
:103BA0000000000C0C00001C04040404040444780D
:103BB000000000C04040404E4850684844EE0000BD
:103BC000000000701010101010101010107C000079
:103BD00000000000000000FE4949494949ED00008D
:103BE00000000000000000DC6242424242E70000A8
:103BF000000000000000003C42424242423C000003
:103C000000000000000000D864424242447840E0D6
:103C1000000000000000001E22424242221E020755
:103C200000000000000000EE3220202020F80000FC
:103C3000000000000000003E42403C02427C0000C8
:103C4000000000000010107C10101010100C00007C
:103C500000000000000000C642424242463B000015
:103C600000000000000000E742242428101000009B
:103C700000000000000000D79292AAAA444400006D
:103C8000000000000000006E2418181824760000C0
:103C900000000000000000E742242428181010E073
:103CA000000000000000007E44081010227E00008A
:103CB00000030404040404080404040404040300CA
:103CC0000808080808080808080808080808080874
:103CD000006010101010100810101010101060006C
:103CE000304C430000000000000000000000000015
:103CF0002800300038004000480050005800000004
:103D0000A800B000B800C000C800D000D800000073
:103D1000000000D000F807D000F00FD0603D000890
:103D2000080000205C00000080260008BC3D000860
:103D300064000020E400020090260008583D0008BE
:103D4000A9360008A5360008AD36000800000000BE
:103D5000D136000800000000757361727400000025
:103D600000000000F0FFFFFF0095BA0A000000000D
:103D7000000000000102030406070809000000001B
:103D80000102030401020304060708090000000001
:103D90000000000000000000000000000000000023
:103DA0000000000000000000000000000000000013
:0C3DB00000000000000000000000000007
:04000005080001AD41
:00000001FF
